S02000006F70656E62746C5F6F6C696D65785F65666D3332673838302E7372656320
S113000060070020C10D00004D1B00004D1B0000C7
S11300104D1B00004D1B00004D1B00004D1B00003C
S11300204D1B00004D1B00004D1B00004D1B00002C
S11300304D1B00004D1B00004D1B00004D1B00001C
S11300404D1B00004D1B00004D1B00004D1B00000C
S11300504D1B00004D1B00004D1B00004D1B0000FC
S11300604D1B00004D1B00004D1B00004D1B0000EC
S11300704D1B00004D1B00004D1B00004D1B0000DC
S11300804D1B00004D1B00004D1B00004D1B0000CC
S11300904D1B00004D1B00004D1B00004D1B0000BC
S11300A04D1B00004D1B00004D1B00004D1B0000AC
S10B00B04D1B00004D1B000074
S11300B8044B9D46C046C046C046C04600F069FE93
S11300C801F09AF960070020890011EB401010F143
S11300D8844002607047DFF89005006810F007015B
S11300E80029012903D9891E012905D908E0C00876
S11300F8C00050F0010003E0C008C00050F0030045
S1130108DFF8641508607047B0FA80F0D0F11F007A
S11301187047DFF854150968DFF85025821ADFF8AC
S113012850359A420DD211F00702921E012A04D8C2
S1130138C908C90051F0030103E0C908C90051F016
S11301480101DFF8282590420BD211F00700801E28
S1130158012804D8C808C00050F0020101E0C90809
S1130168C900DFF8040501607047DFF80805704727
S113017880B5DFF8040500F09EF9C0B2072804D062
S1130188082805D100F0AFFA03E0FFF7EEFF00E01E
S1130198002002BD80B5DFF8E4140968C0B240004D
S11301A831FA00F010F0030000280FD0022806D01E
S11301B802D3032806D00BE000F0CFFA09E000F0E0
S11301C8CFFA06E000F084FA400802E0002000E0DC
S11301D8002002BDDFF8A8140968C90704D4DFF8B1
S11301E8A41409680142FAD1704710B50C00C0F391
S11301F80311012907D0C0F09A80032925D010D310
S1130208042967D093E02000FFF77EFF0400DFF89D
S113021880040068000900012043DFF874140860B2
S113022885E0FFF758FF2000FFF76EFF0400DFF8B2
S113023864040068000900012043DFF858140860CA
S113024800F046FAFFF765FF71E0DFF84C148842C6
S113025808D0DFF84814884215D0DFF848148842DB
S113026823D036E00420FFF7B5FF2000FFF74CFF4A
S11302780400DFF82C040068000900012043DFF8BB
S11302882014086025E00420FFF7A4FF2000FFF7EE
S11302983BFF0400DFF80804006830F0F00050EA7F
S11302A80410DFF8FC13086013E00420FFF792FF42
S11302B82000FFF729FF0400DFF8E403006830F4A6
S11302C84070B4F1100150EA0120DFF8D41308603B
S11302D8FFE72CE0DFF8D013884204D0DFF8CC1312
S11302E8884211D022E04020FFF774FF2000FFF776
S11302F80BFF0400DFF8B80300688008800020437F
S1130308DFF8AC13086011E04020FFF763FF20001A
S1130318FFF7FAFE0400DFF89803006830F03000B5
S113032850EA0410DFF888130860FFE7FFE710BD00
S113033870B50C000021C0F30322D2B2012A09D0FF
S113034829D3032A19D015D3052A1DD018D3062A70
S11303581ED020E0DFF83853C0F30436002902D059
S11303680800FFF737FFE4B2220031002800FFF746
S1130378ABFE70BDDFF83C53EEE7DFF83C53EBE728
S1130388DFF838530121E7E7DFF834531021E3E7B6
S1130398DFF83053E0E7ECE780B510F47810002874
S11303A824D0B0F5003F24D0B0F5802F2AD0B0F582
S11303B8C02F2AD0B0F5002F2BD0B0F5202F32D083
S11303C8B0F5402F39D0B0F5602F41D0B0F5901F6B
S11303D851D0B0F5A01F52D0B0F5B01F59D0B0F528
S11303E8C01F60D0B0F5D01F60D062E000F07BF988
S11303F860E000F078F9DFF89812096811F00F014D
S1130408C84057E000F064F954E00020FFF7C2FE4A
S113041850E00020FFF7BEFEDFF88412096811F0EF
S11304280F01C84046E00020FFF7B4FEDFF8701261
S11304380968C1F30311C8403CE00020FFF7AAFE95
S1130448DFF85C120968090A11F00301C84031E0B9
S11304580020FFF79FFEDFF848120968090A11F027
S11304680301C840DFF86012096811F00701491C4C
S1130478B0FBF1F01EE00120FFF78CFE1AE001202A
S1130488FFF788FEDFF82812096811F00301C84055
S113049810E00120FFF77EFEDFF814120968C1F3AB
S11304A80111C84006E0FFF763FE03E0FFF75DFEB5
S11304B800E0002002BD012110F00F00012806D041
S11304C836D303282DD018D304282FD030E0DFF8F2
S11304D8BC01006810F47050B0F5006F09D0B0F595
S11304E8805F04D0B0F5005F05D1022104E0032148
S11304F802E0042100E005211BE0DFF88001006828
S113050810F00300012804D009D3032805D002D32E
S113051805E0032104E0022102E0062100E00121B4
S113052807E0DFF858010068012102E0072100E034
S113053800210800C0B2704738B50324032310F023
S11305480F000200521E03D0521E012A27D956E07A
S1130558C9B2022906D021D3042919D015D30529F3
S113056819D01BE004240023012201211800C0B281
S113057800F046F8FFF7AFFD4348046000F00CF9BB
S113058800F0A6F8FFF7C5FD39E003240123EBE7E3
S113059802240223E8E701240323E5E72FE00228E5
S11305A801D1002400E00224C9B2012906D002299D
S11305B80FD0032914D0062919D01FE000202F4991
S11305C809680322A2409143A04008432B490860CC
S11305D815E001220121002000F012F80220EEE7C4
S11305E801220121012000F00BF80120E7E7012294
S11305F802213148FFF768FD0320E0E7FFE731BD3A
S113060810B5C0B2002821D0022813D01AD3042868
S113061814D022D2012302240220C9B200291DD0F9
S11306282A490B60D2B2002A1AD018490968014233
S113063816D1FAE7042308240820EEE7102320241F
S11306482020EAE7402380248020E6E74FF48073E3
S11306584FF400744FF40070DFE703E01B480460B4
S113066800F09AF810BD000004000C400124F400C6
S11306780024F400809FD5000400180028800C4052
S113068854800C4050800C4024800C402C800C403A
S113069808800C4004800C403004080030140A0020
S11306A868800C4030000C0040051400401516000A
S11306B870800C4044800C4040800C4058800C40B2
S11306C860800C4078800C407C800C4020800C407A
S11306D880B500F008F82449096811F00F01C840F2
S11306E82249086002BD2248006810F47050B0F531
S11306F8006F0BD0B0F5805F05D0B0F5005F08D16E
S11307081C48006827E04FF4004024E01A480068B9
S113071821E01A48006810F4E060002818D0B0F509
S1130728807F13D0B0F5007F0ED0B0F5407F09D09C
S1130738B0F5806F04D0B0F5A06F0BD110480AE073
S1130748104808E0104806E0104804E0104802E0A9
S1130758104800E00020704770474FF4004070478D
S1130768044800687047000004800C4054060020C8
S11307782C800C40700100206C0100200C800C407F
S1130788003FAB01406F4001809FD500C0D8A7004F
S1130798C0CF6A0040420F0002480349096801803B
S11307A870470000580600202C800C40DFF800F049
S11307B889000020DFF800F00100002080B500F077
S11307C845FADFF878045FF0FF310160DFF8700460
S11307D85FF0FF31016001BD70B504000D00160023
S11307E8200000F0C8F9FF2805D02819401E00F0A1
S11307F8C2F9FF2801D1002019E0600A4FF4007102
S11308084843DFF840140968884208D12B009BB29A
S113081832002100DFF8280400F0E9F807E02B0093
S11308289BB232002100DFF8140400F0E0F870BD38
S113083870B504000D00200000F09DF90600281989
S1130848401E00F098F9F6B2FF2E02D0C0B2FF287D
S113085801D1002005E00100C9B23000C0B200F0A7
S113086849F970BD80B500200090DFF8D403006812
S113087810F1010F01D1012037E00098DFF8C0130F
S11308884968081800900098DFF8B41389680818B4
S113089800900098DFF8A813C96808180090009819
S11308A8DFF89C130969081800900098DFF8901382
S11308B84969081800900098DFF8841389690818B2
S11308C800900098DFF87813C96908180090009818
S11308D8C04300900098401C009000AA0421DFF84F
S11308E864030068B830FFF777FF02BD0020DFF823
S11308F85413096809680818DFF84813096849682F
S11309080818DFF84013096889680818DFF83413F1
S11309180968C9680818CB49096809690818C949E0
S1130928096849690818C749096889690818C549D7
S11309380968D1F8B8100818002801D1012000E08E
S11309480020704780B5BE48006810F1010F06D03A
S1130958BB4800F091F8002801D100200EE0B74808
S1130968006810F1010F06D0B44800F085F800289B
S113097801D1002002E000F07AF9012002BD80B51F
S11309884FF40072B1FBF2F303FB1213002B01D0F6
S113099800200BE002688A4201D1012006E00160D0
S11309A84FF40072001D00F089F9012002BD38B52A
S11309B804000D00A248844208D1A04C290020005C
S11309C8FFF7DDFF002810D100200FE09D480068E4
S11309D8854203D19A4C9B480568EFE7200000F054
S11309E84BF80028EAD1002000E0200032BD2DE9B0
S11309F8F04104000F0015001E00780A4FF400713E
S1130A0801FB00F8206810F1010F07D141462000CE
S1130A18FFF7B5FF002801D100202BE020684045EE
S1130A2808D041462000FFF7C2FF0400002C01D182
S1130A3800201FE02068381A0019071D00F054F937
S1130A48201D381A4FF4007188420AD308F2002195
S1130A582000FFF7ACFF0400002C01D1002009E0BE
S1130A68271D287838707F1C6D1C761EB6B2012E9F
S1130A78E4D20120BDE8F081F8B505000124286816
S1130A8800F079F8C0B2FF2801D100201DE000264B
S1130A9800E0761C802E16D2286810EB860715EB2A
S1130AA886004068009000F01FF9042200A938006D
S1130AB8FFF77CFE002801D0002404E03868009980
S1130AC88842E6D000242000C0B2F2BD5E48007817
S1130AD8C0B2472802D0C0B2492802D14FF40070EE
S1130AE807E0C0B2482802D14FF4805001E04FF427
S1130AF800607047F8B506000C00E4B2F6B2B442E0
S1130B0801D2002036E04F48007AF6B2864205D377
S1130B184C4890F8B000E4B2A04201D2002029E089
S1130B28FFF7D4FF05003000C0B200F04EF806000D
S1130B382000C0B200F049F807002000C0B200F05D
S1130B4861F8C019401E801B401CB0FBF5F4002757
S1130B5800E07F1CBFB2A4B2A7420AD200F0C4F8D6
S1130B68BFB205FB0760FFF725FE0028F1D000207F
S1130B7800E00120F2BD38B50400002500E06D1C3A
S1130B88EDB20F2D1FD200F0AFF8EDB20C202D49B5
S1130B9800FB051000688442F1D3EDB20C2029490A
S1130BA800FB05100068EDB20C21264A01FB052163
S1130BB8496808188442E2D2EDB20C20214900FBAE
S1130BC80510007A00E0FF2032BD38B50400002586
S1130BD800E06D1CEDB20F2D11D200F085F8EDB2D6
S1130BE80C20184900FB0510007AE4B2A042F0D1A9
S1130BF8EDB20C20134900FB0510006801E05FF01A
S1130C08FF3032BD38B50400002500E06D1CEDB29C
S1130C180F2D11D200F068F8EDB20C20094900FB41
S1130C280510007AE4B2A042F0D1EDB20C200549D7
S1130C3800FB0510406800E0002032BD740100206C
S1130C4878030020D8190000FE81E00F10480068DE
S1130C5850F001000E4908600E4841F671310160F8
S1130C680B48006840084000094908607047084874
S1130C78006850F001000649086006480021016038
S1130C8803480068400840000149086070470000B4
S1130C9808000C403C000C4080B500F032F80028F5
S1130CA809D000F06EF804484FF40051016042F294
S1130CB804000068804701BD08ED00E070B5040039
S1130CC80D00160005E0287820706D1C641C00F0E7
S1130CD80BF83000461E80B20128F4D270BD80B5EE
S1130CE800F06AF801BD7047704780B5FFF766FDEC
S1130CF801BD80B5FFF770FD02BD80B5FFF798FD13
S1130D0802BD80B5FFF7F2FD02BD80B5FFF7AAFD6D
S1130D18002801D1002001E0FFF714FE02BD10B441
S1130D2850F8041B81B102681218001D50F8043BE6
S1130D38DC0744BFA9F10104E31852F8044B43F853
S1130D48044B091FF9D1EBE710BC704780B500A824
S1130D5814490A88028000F03BF800F06FFA124840
S1130D680078012802D100A800F05CF801BD80B524
S1130D780E4800F0CEFA012802D10C4800F052F8CF
S1130D8801BD704780B5C9B200F099FA00F044F883
S1130D9801BD054801210170704703480021017015
S1130DA87047000016140000600700200C0600209D
S1130DB880B500F028F802BD044B9D46C046C046E5
S1130DC8C046C046FFF7E9FF00F016FB60070020A5
S1130DD8DFF8240400210170DFF81C040021816479
S1130DE8DFF81404002180F84310DFF80C04002114
S1130DF8A0F84410DFF8000400218170DFF8F8033C
S1130E08002141707047DFF8F0030078002801D111
S1130E18002000E001207047DFF8DC03002180F89F
S1130E284310704780B50178FF2918D100F08BF87A
S1130E38DFF8C40390F84300012802D1102000F021
S1130E4878F8DFF8B403012180F84310DFF8A80329
S1130E58B0F94410DFF8A40300F053F801BDDFF83B
S1130E689813097801294BD10178C92932D0CC29A2
S1130E783FD0CF293AD0D0292FD0D12933D0D22965
S1130E882ED0F32917D0F4290FD0F5290AD0F62942
S1130E980ED0FA2912D0FC2913D0FD2914D0FE292A
S1130EA815D029E000F0CDF8C2E700F0E9F8BFE773
S1130EB800F0BCF8BCE700F005F9B9E700F09EF8CB
S1130EC8B6E700F095F8B3E700F07AF8B0E700F079
S1130ED868F8ADE700F027F9AAE700F03EF9A7E7BC
S1130EE800F007F9A4E700F066F9A1E700F077F944
S1130EF89EE700F08BF99BE7202000F01AF897E7AB
S1130F08ACE780B589B2FFF73DFF01BD10B40023FB
S1130F1802E00478E318401C0C00611E002CF8D190
S1130F28DBB21360012010BC7047B3480021417044
S1130F387047B149FE22CA70AF490871AE48022110
S1130F48A0F84410704710B50400FFF7EEFFAA4854
S1130F5801210170A848FF21C170A748002101712F
S1130F68A548007950F01000A3490871A24800214F
S1130F784171A148A049497941719F484021817133
S1130F889D484021C1719C48002101729A48012161
S1130F98417299480121817297480821A0F84410A8
S1130FA810BD10B50400944800210170FFF7BDFF7F
S1130FB89148FF21C17090480121A0F8441010BD48
S1130FC88D49FF22CA708C4900220A718A498A4ACB
S1130FD852784A71884900228A7187490022CA7165
S1130FE8854900220A7284490622A1F844207047E0
S1130FF810B504000020FFF79CFF10BD7E49FF22B6
S1131008CA707D497E4A8A647B4900220A717A49FA
S113101800224A71784900228A7177490722C1F867
S1131028072075490822A1F8442070477249FF2215
S1131038CA707149406888646F480121A0F8441057
S1131048704710B504006078402803D32220FFF7C6
S113105870FF14E0627892B26748816C6948FFF7C0
S11310682DFE6548FF21C1706348806C61780818BB
S1131078614988646078401C5F49A1F8440010BD48
S113108810B504006078402803D32220FFF751FFED
S113109817E0594861688164627892B25648816C55
S11310A85848FFF70BFE5448FF21C1705248806C22
S11310B861780818504988646078401C4E49A1F842
S11310C8440010BD80B54C49FF22CA704E4A41689D
S11310D84948806CFFF71AFF4749087146480021C0
S11310E8417145480021817143480821A0F8441002
S11310F801BD4149FF22CA703F4900220A713E4995
S113110800224A713C4940228A713B490022CA7133
S1131118394900220A72384900224A72364907229C
S1131128A1F84420704780B5421C3F213248806CA6
S1131138FFF7DFFD002803D13120FFF7FAFE0BE0AB
S11311482D48FF21C1702C48806C3F302A4988649F
S113115829480121A0F8441001BD10B504006078A5
S11311683F2803D32220FFF7E4FE23E02248FF218F
S1131178C17021480121A0F844106078002807D1E3
S1131188FFF7C3FD002802D13120FFF7D2FE11E09A
S1131198A21C61781848806CFFF7ABFD002803D1C6
S11311A83120FFF7C6FE05E01348806C6178081803
S11311B81149886410BD80B541680F48806CFFF7F9
S11311C89CFD002803D13120FFF7B3FE06E00A484E
S11311D8FF21C17008480121A0F8441001BD10B5D1
S11311E80400FFF77CFD0448FF21C1700248012177
S11311F8A0F8441010BD00007C0500207F050020E5
S1131208681B0000800500208305002080B531207C
S1131218FFF78FFE01BD50F8041B61B150F8042B91
S1131228D30744BFA9F101039A18002342F8043BE9
S1131238091FFAD1EFE770474163704700B585B0DD
S113124800A85F49102200F0E3F801215D48FFF788
S11312586FF8012304220621022000F016F9002366
S113126801220721022000F010F901215648FFF756
S11312785FF802215548FFF75FF901215448FEF74A
S1131288B4FF01215248FFF753F800208DF80000FD
S113129800A9504800F0ADF94FF4165200214D480A
S11312A800F065F94C480321016004214948FFF71F
S11312B8C3FF0521474800F081F905B000BD70B5AA
S11312C804000D00EDB2412D03D36821434800F01A
S11312D8C7F92800C0B200F05DF8012803D06B21DB
S11312E83E4800F0BDF900260CE0FFF7FDFCB6B25D
S11312F8305D00F04FF8012803D07321374800F01F
S1131308AFF9761C2800C0B2B6B280B28642ECD3DC
S113131870BD10B504003248007800280CD131485B
S113132800F02AF8012805D12D48012101702E4822
S113133800210170002010BD2B480078294940186D
S1131348401C00F019F80128F4D127480078401C03
S11313582549087024480078224909788842E9D147
S11313682148027892B221492000FFF7A7FC1C48C3
S1131378002101700120DEE710B5040000201C499B
S11313880968490704D5134800F056F9207001206C
S1131398C0B210BD80B517490968C90601D4002038
S11313A80CE00100C9B20B4800F04CF901E0FFF76A
S11313B89BFC10480068C006F9D5012002BD000056
S11313C83C1B000000C202000023040003001200BA
S11313D8401516000044084054440840D41A00003C
S11313E85E060020C80500205D060020C90500200F
S11313F82C4408400844084000F03EF9002801D075
S113140800F03CF9002000F0BEF900F057FAFF00A4
S1131418103A07D330B4B1E83810103AA0E83810BD
S1131428F9D230BC530724BFB1E80810A0E808106B
S113143844BF51F8043B40F8043BD20724BF31F8B9
S1131448022B20F8022B44BF0B7803707047083A2C
S113145807D3B1E80810083A40F8043B40F804CB35
S1131468F7D25307E4E70000C0B224223B4B02FB47
S11314780032126892089200C9B21143C0B2242201
S1131488364B02FB00300160704770B4D2B2002AB8
S113149812D0002B08D0C0B22424304D04FB0054D1
S11314A801258D40256107E0C0B224242B4D04FB9F
S11314B8005401258D406561082919D2C0B224243D
S11314C8264D04FB005464680F250E00F6B2B600DE
S11314D8B540AC43D2B20D00EDB2AD0012FA05F539
S11314E82C43C0B224251D4E05FB00656C601AE030
S11314F8C0B22424194D04FB0054A4680F250E001F
S1131508083EF6B2B600B540AC43D2B20D00083D71
S1131518EDB2AD0012FA05F52C43C0B224250F4EE6
S113152805FB0065AC60D2B2002A14D1002B09D0A7
S1131538C0B22422094B02FB0030012212FA01F145
S1131548016108E0C0B22422044B02FB00300122EE
S113155812FA01F1416170BC70470000006000405C
S1131568026CD20702D4426C0A42FCD1704738B5E7
S113157804001500002906D10C4884420ED10C48F9
S1131588FEF70AFF01004801B0FBF5F5203DED0028
S113159804212000FFF7E4FFE56031BD05488442DB
S11315A801D10548ECE7F8E70000000000400840D6
S11315B840051400004408404015160038B50400DE
S11315C8C9B2CD4315F005056D00C9B20D4302211A
S11315D82000FFF7C5FF656031BDC9B2002905D0F9
S11315E8416C0029FCD10121016401E0002101645E
S11315F8704738B504000D0002212000FFF7B0FF42
S11316080A20606001212000FFF7E7FF206830F01E
S11316181C00297B0843697B0843A97B0843206095
S1131628AA6869682000FFF7A2FF28786060002193
S11316382000FFF7D2FF31BD81688906FCD5C06957
S1131648C0B2704738B504000D00A068C006FCD5C8
S113165840212000FFF784FFEDB2A56231BD0000F0
S113166880B5034A106003480160FFF73DFBFCE7BF
S11316784C060020500600200120704710B5084988
S113168879441C31074C7C441A34A14206D0081D05
S11316980A68511888470146A142F8D110BD00BF15
S11316A8700400009004000080B568480168080EC2
S11316B800280DD16648026832F07002026065485D
S11316C80268D200D2080260026872F060620260A6
S11316D8080E042813D25F48016831F4FC510160F4
S11316E85D48002101605D48002101605C480021DB
S11316F801605C48002101605B480021016000A88A
S113170800F0DEF89DF80000012811D19DF80100D1
S1131718002804D15048016851F0020101609DF885
S11317280100022804D24D48016851F0010101600A
S11317384E4801684E48814224D24848016851F411
S1131748904101604B480068000410F0FE4149488C
S1131758006810F07F0051EA00414648006810F420
S1131768FE4001434348006810F07F0001434248AB
S1131778016042484249096801603848016831F407
S11317889041016001BD80B500F005F800F0AEF8A5
S113179800F0B6F8FCE780B5FEF7DEFFFFF784FF3C
S11317A8012201210020FEF72BFF2B48006850F08E
S11317B80F00294908602948006840F47F4050F028
S11317C8FF002649086000212E48FEF7B1FD0021DC
S11317D82D48FEF7ADFD00212C48FEF7A9FD002198
S11317E82B48FEF7A5FD00212A48FEF7A1FD00219C
S11317F82948FEF79DFD00212848FEF799FD0021A0
S11318082748FEF795FD00212648FEF791FD0021A3
S11318182548FEF78DFD00212448FEF789FD0021A7
S11318282348FEF785FD00212248FEF781FD0021AB
S11318382148FEF77DFD0123052209210120FFF738
S113184824FE02210120FFF70FFE01BDFC81E00FF9
S11318580CA00C4020600C4040800C4044800C409C
S113186858800C4060800C4078800C40F081E00F78
S113187800BA8A4CB481E00F342000402C40004068
S1131888C881E00F000304000013040000330400BF
S113189800A202000002020000120200002202005C
S11318A800320200007202000082020000B202004C
S11318B800E2020000F2020000D2020000F028B8A0
S11318C80749096811F03F0101700649096811F0D8
S11318D8F001054A1268C2F30312114341707047BC
S11318E8E0FF0FE0E8FF0FE0ECFF0FE080B5FFF743
S11318F8FAF900F013F8FFF7F8F9FFF727FA01BD32
S113190880B5FFF7F1F9FFF732FA00F010F801BDDE
S11319180746384600F022F8FBE7000080B50E4879
S11319280121017000F024F800F001F801BD80B530
S1131938FFF73EFA01280ED00748007801280AD19B
S113194800F038F8322806D303480021017000F06B
S113195820F8FFF7A1F901BD5C06002080B5C04658
S1131968C046024A11001820ABBEFBE7260002005D
S113197880B500F00EF8124843F2AF6101601148D7
S113198800210160104805210160002000F00FF8D3
S113199801BD0D480021016070470B480068C00371
S11319A804D50A480088401C08490880704707493C
S11319B80880704780B5FFF7F0FF0448008802BD2F
S11319C814E000E018E000E010E000E05A0600200F
S11319D8002000000020000001000000004000007A
S11319E80020000002000000006000000020000049
S11319F80300000000800000002000000400000034
S1131A0800A00000002000000500000000C0000045
S1131A18002000000600000000E000000020000094
S1131A28070000000000010000200000080000007A
S1131A38002001000020000009000000004001000F
S1131A48002000000A0000000060010000200000DF
S1131A580B00000000800100002000000C000000C2
S1131A6800A00100002000000D00000000C00100DB
S1131A78002000000E00000000E00100002000002B
S1131A880F000000443A5C7573725C6665617365A7
S1131A98725C736F6674776172655C4F70656E42D1
S1131AA84C545C5461726765745C536F75726365FA
S1131AB85C41524D434D335F45464D33325C494199
S1131AC8525C766563746F72732E6300443A5C7576
S1131AD873725C6665617365725C736F6674776153
S1131AE872655C4F70656E424C545C5461726765F4
S1131AF8745C536F757263655C41524D434D335F3B
S1131B0845464D33325C756172742E6300000000E3
S1131B1807F7FFFFEC040000740100200000000038
S1131B28FFF1FFFF740100004000000000000020E6
S1131B3800000000050000000000000080250000EF
S1131B480000000080B540210148FFF789FD01BD70
S1131B588C1A0000C046C046C046C046FFF74CFC7D
S1131B684F70656E424C54005449554A126852F0FD
S1131B780102534B1A60534A106053480122026011
S1131B8852480068400708D54D480068400840009E
S1131B984B4908605FF0FF3029E04C480068800733
S1131BA808D54748006840084000454908607FF068
S1131BB801001CE044480222026000E0491E434838
S1131BC80068C00701D50029F8D1002908D13C488C
S1131BD80068400840003A4908607FF0020006E0C7
S1131BE837480068400840003549086000207047BD
S1131BF830B4334B1B6853F00103314C236093100A
S1131C08002200E0521C9A424FDA10EB82042D4D58
S1131C182C602D4C012525602C4C2468640708D5BC
S1131C282748006840084000254908605FF0FF30F5
S1131C3842E0264C2468A40708D5214800684008D7
S1131C4840001F4908607FF0010035E01B4C00E0AC
S1131C58641E1E4D2D682D0701D4002CF8D1002CCC
S1131C6808D11748006840084000154908607FF00B
S1131C78020021E051F82240154D2C60124C082531
S1131C8825600E4C00E0641E104D2D68ED0701D54B
S1131C98002CF8D1002CB5D1094800684008400050
S1131CA8074908607FF0020006E00548006840081C
S1131CB8400003490860002030BC704780969800B3
S1131CC808000C4010000C400C000C401C000C4098
S10F1CD818000C400048E80100800000E7
S9031B5D84
